:100000000C9465000C94F7010C9401020C9482008E
:100010000C9482000C9482000C9482000C94820058
:100020000C9482000C9482000C9482000C94820048
:100030000C9482000C94ED010C9482000C948200CC
:100040000C9482000C9482000C9482000C94820028
:100050000C940B020C9482000C9482000C9482008D
:100060000C9415020C9482000C9482000C94820073
:100070000C9482000C9482000C9482003C407C40E2
:100080007C003C407C407C003C407C407C0000602C
:100090006000000038545454480038545454480008
:1000A0007C08040404003844444444004464544C30
:1000B0004400006060000000384444444400384478
:1000C000444438007C047C04780011241FBECFEF28
:1000D000D8E0DEBFCDBF11E0A0E0B1E0ECE4F5E098
:1000E00002C005900D92A230B107D9F715E0A2E049
:1000F000B1E001C01D92A13FB107E1F70E94730278
:100100000C94A4020C9445024398409827E030E0F8
:10011000482F50E0CA01022E02C0959587950A9497
:10012000E2F780FF02C0419A01C04198409A40988E
:10013000215030408FEF2F3F380761F7439A0895E1
:1001400042980E9484000895429A0E948400089573
:10015000459A0000000000000000000000000000C0
:100160000000449800000000449A81E20E94A00030
:10017000809100010E94A00083E10E94A00080E223
:100180000E94A0008CE00E94A00080E40E94A000D9
:1001900080E80E94A00008954498409841984298B1
:1001A000439845984698089581E20E94A000809166
:1001B00000010E94A00080E20E94A00008951F9309
:1001C000162F80680E94A0001774812F80640E94FF
:1001D000A0001F910895CF93DF9380E060E00E941C
:1001E000DF00C0E0D0E080E00E94A400219681E022
:1001F000C83FD807C1F780E060E00E94DF00DF91D0
:10020000CF910895BF92CF92DF92EF92FF920F931A
:100210001F93CF93DF9329E4E22E25E0F22EC3EF64
:10022000D4E001E091E0C92ED12C8FE0B82EF70187
:10023000808191810090010102C0969587950A9472
:10024000E2F7182F802F60E00E94DF0080E00E941C
:10025000A400802F61E00E94DF0080E00E94A400E3
:10026000802F62E00E94DF0080E00E94A400802FC7
:1002700063E00E94DF0080E00E94A400888182FF8A
:1002800017C0FB2DF11B1F2FF83078F0802F61E095
:100290000E94DF00812F90E00897960102C0220F94
:1002A000331F8A95E2F7C9011EC0802F60E013C09A
:1002B000183078F0802F63E00E94DF00812F90E0FB
:1002C0000897F60102C0EE0FFF1F8A95E2F7CF01F3
:1002D0000AC0802F62E00E94DF00C60102C0880FC2
:1002E000991F1A95E2F70E94A4000F5F22E030E008
:1002F000E20EF31E2196043509F099CFDF91CF91DC
:100300001F910F91FF90EF90DF90CF90BF900895D5
:10031000FF920F931F932091EE04A22FB0E08091E3
:10032000020163E00E949802F82EFD01EA5FFE4F91
:1003300080838091030160E30E949802082FA650F9
:10034000BD4F8C932F5F2093EE042150253610F083
:100350001092EE04E091EE04F0E0DF01A650BD4FF4
:10036000EA5FFE4F80816C910E94DF0080E00E9476
:10037000A400109103018F2D602F0E94DF00812FB8
:1003800066E00E949802877021E030E0922F01C061
:10039000990F8A95EAF7892F0E94A400F092040130
:1003A000009305011F910F91FF900895CF93DF9364
:1003B00082E065E00E94DF00CCE7D0E006C0FE01ED
:1003C0002196E4918E2F0E94A40080E0C93CD807BA
:1003D000B1F7DF91CF91089508951F920F920FB654
:1003E0000F9211240F900FBE0F901F9018951F921F
:1003F0000F920FB60F9211240F900FBE0F901F9007
:1004000018951F920F920FB60F9211240F900FBEE6
:100410000F901F9018951F920F920FB60F921124F4
:100420000F900FBE0F901F9018951F920F920FB64E
:100430000F9211248F939F93909179008091EF04F4
:10044000882381F480917C00816080937C0080917E
:100450007A00806480937A009093020181E0809317
:10046000EF040CC080917C008E7F80937C00909381
:1004700003011092EF0481E08093F0049F918F912B
:100480000F900FBE0F901F9018951F920F920FB6EE
:100490000F9211240F900FBE0F901F9018951F936D
:1004A000F894A8952FE088E190E00FB6F894A8950D
:1004B000809360000FBE20936000A89587B18F6085
:1004C00087B93C9A87B1806687B91FEF17B90E9438
:1004D000A8000E94EB000E94D60112B915B914B908
:1004E0001AB91F9108950E944F02A895A8952A98BD
:1004F0002898000000000000289A2A9A2B98299832
:10050000000000000000299A2B9A2A9800000000A1
:10051000000080B1809302012A9A2B98000000000D
:10052000000080B1809303012B9A0E948801DECFE6
:10053000991B79E004C0991F961708F0961B881F35
:0C0540007A95C9F780950895F894FFCFD4
:02054C00CD06DA
:00000001FF
